:0400000019EF26F0DE
:1000080000C016F001C015F06F0084FF17F06F00F4
:1000180088FF18F0390193AF13D0A3AF11D03C0E6D
:10002800B76EB00EB66E194A1A2A000E006E1A5034
:10003800005C02E11950090802E2BB763184A39FF3
:10004800A3A76FD093A76DD014EC25F000C004F1DE
:100058003D01F9AB0FD0F99B010E01011B25006E84
:10006800000E1C21016E00C01BF101C01CF16F00C5
:10007800A0F704F13D01F9A70FD0010E01011B25DE
:10008800006E000E1C21016E00C01BF101C01CF1A6
:1000980014EC25F000C004F1010104510D0A07E039
:1000A8003550000802E134504F0801E31AD0010E20
:1000B800116F000E126FB20E3C24E16E000E3D204F
:1000C800E26E6F0087FFE1FF6F008BFFE2FFE66AD9
:1000D800390193973CC034F03DC035F03C6A3D6A25
:1000E80020D00101116B126BB20E3C24E16E000EA0
:1000F8003D20E26E6F0087FFE1FF6F008BFFE2FF9C
:10010800600013F4E6FF3CC034F03DC035F0010E4A
:100118003C24006E000E3D20016E00C03CF001C082
:100128003DF016C000F015C001F060005FF0E1FF7F
:08013800600063F0E2FF11001A
:0C014000000E3D01F9BF010E006E120020
:0C014C00000E3D01E1BF010E006E12002C
:04015800F9DF1200B9
:04015C00F1DF1200BD
:100160000B820BAEBAEF00F003680268016800680A
:080170000A360232FF0E1200F4
:080178000AAE029E000E120007
:10018000EBDF005202E10000FBD76000ABF5D2FDCF
:0201900012005B
:0E019200026A016A006A086A036A000E12001F
:1001A000DDDF005202E10000FBD76000ABF5EAFDA5
:0201B00012003B
:1001B2000B840BAEE4EF00F0010E036E026A016ADB
:0A01C200006A0A360232FF0E120036
:0E01CC00550E3A01BF6FAA0EBF6FBF81120021
:0801DA0069C16AF1E0DF1200C7
:0801E20069C16AF1CCDF1200D3
:0E01EA00550E3A01BF6FAA0EBF6FBF911200F3
:1001F8000CB03EEF01F00CA2E4EF01F00E6A000E25
:10020800026455EF01F0F00E0214D8A420EF01F0BB
:10021800023A01380F0B02260138F00B016E003844
:100228000F0B01260038F00B006E08380F0B002664
:100238000838F00B086E0E84D89002BE39EF01F032
:1002480008360036013602360E2A02BE39EF01F0B2
:1002580008360036013602360E2A02BE39EF01F0A2
:1002680008360036013602360E2A0E500364DAEFDD
:1002780001F0035E0BBC08AEDFEF01F0D880800E02
:1002880008640030000E002201220222D8A0DFEF0D
:1002980001F0023201320032034AE4EF01F0DFEFED
:1002A80001F001C002F000C001F008C000F0086AC7
:1002B800000E0E8602648CEF01F0F00E0214D8A432
:1002C80074EF01F0023A01380F0B02260138F00BE7
:1002D800016E00380F0B01260038F00B006E0E84FB
:1002E800D89002BE39EF01F00036013602360E2AE8
:1002F80002BE39EF01F00036013602360E2A02BE80
:1003080039EF01F00036013602360E2A39EF01F0D6
:1003180001C002F000C001F0006A000E0E960E88BF
:100328000264B9EF01F0F00E0214D8A4A4EF01F0B2
:10033800023A01380F0B02260138F00B016E0E84C9
:10034800D89002BE39EF01F0013602360E2A02BEFD
:1003580039EF01F0013602360E2A02BE39EF01F0FC
:10036800013602360E2A39EF01F001C002F0016AA7
:10037800000E0E860264E9EF01F0F00E0214D8A414
:10038800C8EF01F0023A0E84D89002BE39EF01F0AE
:1003980002360E2A02BE39EF01F002360E2A02BEDC
:1003A80039EF01F002360E2A39EF01F0010E0C6E1A
:1003B800FCDEECEF01F0020E0C6EDADEECEF01F081
:1003C800040E0C6EC9DEECEF01F0080E0C6EDDDEDB
:0203D800120011
:0803DA0069C16AF1D0DE1200D6
:0803E20069C16AF1DCDE1200C2
:1003EA00086A096A000E076203647DEF02F0025090
:1003FA0006180A6E075003267E0ED8A00BEF02F0ED
:10040A00035ED8B081EF02F00FEF02F0035ED8A0CE
:10041A0085EF02F0028E068E02C00EF001C00BF0CC
:10042A0000C00DF0005004026F00D0FF0CF0015024
:10043A0005026F00D0FF00F06F00CCFF08F0040245
:10044A00F3500C26F4500822000E00220D5005022B
:10045A00F3500C26F4500822000E00220250040227
:10046A00F3500826F450002202500502016A000ED9
:10047A000122F3500026F45001220D500602F350D7
:10048A000826F4500022026A000E012202220B50B2
:10049A000602F3500026F4500122000E02220E50EA
:1004AA000602F3500126F450022202BE65EF02F062
:1004BA0008360036013602360306D8B485EF02F054
:1004CA0078EF02F0D880800E08640030000E002217
:1004DA0001220222D8A078EF02F002320132003261
:1004EA00034A81EF02F00AAE029E000E87EF02F085
:1004FA00010E4ADE87EF02F0020E2DDE87EF02F0D0
:06050A00040E52DE120097
:080510000B6A0B86FF0E1200BE
:100518000134083609360450085E0550D8A0053C59
:10052800095E003601360F0E0C6E013408360936A6
:10053800045000A006D0085E0550D8A0053C095E0E
:1005480005D008260550D8B0053C092600360136E6
:100558000C2EEBD700B006D0045008260550D8B0B2
:08056800053C09260000120009
:100570000D6A086A0050D8B4000C04180A6E0ABE4E
:100580000D1E0B6A04AE02D0041E042A00AE02D077
:10059000001E002A005004100A6E0ABE1FD004502C
:1005A000085E003600340836045008260036060E71
:1005B0000C6E00340836045000B0085E00A0082617
:1005C00000360C2EF6D700A008260BB015D00DAEC5
:1005D000000C001E002A081E082A000C04AE09D0D8
:1005E00000BE04D00050086E006AF1D7006A002AED
:1005F000000C001E0B2AD3D7082A0450085CD8A48C
:0E060000E6D7086A002A00AEE2D7FF0C12000F
:10060E00086A080E0C6E003408360450085ED8B026
:0E061E0002D00826D89000360C2EF5D7120018
:10062C0001016551170802E2006A0FD36651000AF6
:10063C00D8A4B1D0685301E0D2DD60D060009FF542
:10064C0000FAA5D060009FF501FAA1D060009FF5DB
:10065C0002FA9DD060009FF503FA99D060009FF5D7
:10066C0004FA95D060009FF505FA91D060009FF5D3
:10067C0006FA8DD060009FF507FA89D060009FF5CF
:10068C0008FA85D060009FF509FA81D060009FF5CB
:10069C000AFA7DD060009FF50BFA79D060009FF5C7
:1006AC000CFA75D060009FF50DFA71D060009FF5C3
:1006BC000EFA6DD060009FF50FFA69D060009FF5BF
:1006CC0010FA65D060009FF511FA61D060009FF5BB
:1006DC0012FA5DD060009FF513FA59D060009FF5B7
:1006EC0014FA55D060009FF515FA51D060009FF5B3
:1006FC0016FA4DD060009FF517FA49D001016551EB
:10070C00000A9CE06551010A9DE06551020A9EE0D9
:10071C006551030A9FE06551040AA0E06551050A82
:10072C00A1E06551060AA2E06551070AA3E06551F4
:10073C00080AA4E06551090AA5E065510A0AA6E079
:10074C0065510B0AA7E065510C0AA8E065510D0A2A
:10075C00A9E065510E0AAAE065510F0AABE065519C
:10076C00100AACE06551110AADE06551120AAEE019
:10077C006551130AAFE06551140AB0E06551150AD2
:10078C00B1E06551160AB2E06551170AB3E00101F8
:10079C00685301E015DD01016651010AD8A452D15C
:1007AC00685301E01CDDA4D0600097F5C0FA45D178
:1007BC00600097F5C1FA41D1600097F5C2FA3DD1BE
:1007CC00600097F5C3FA39D1600097F5C4FA35D1BA
:1007DC00600097F5C5FA31D1600097F5C6FA2DD1B6
:1007EC00600097F5C7FA29D1600097F5C8FA25D1B2
:1007FC00600097F5C9FA21D1600097F5CAFA1DD1AE
:10080C00600097F5CBFA19D1600097F5CCFA15D1A9
:10081C00600097F5CDFA11D1600097F5CEFA0DD1A5
:10082C00600097F5CFFA09D1600097F5D0FA05D1A1
:10083C00600097F5D1FA01D1600097F5D2FAFDD09E
:10084C00600097F5D3FAF9D0600097F5D4FAF5D09B
:10085C00600097F5D5FAF1D0600097F5D6FAEDD097
:10086C00600097F5D7FAE9D0600097F5D8FAE5D093
:10087C00600097F5D9FAE1D0600097F5DAFADDD08F
:10088C00600097F5DBFAD9D0600097F5DCFAD5D08B
:10089C00600097F5DDFAD1D0600097F5DEFACDD087
:1008AC00600097F5DFFAC9D0600097F5E0FAC5D083
:1008BC00600097F5E1FAC1D0600097F5E2FABDD07F
:1008CC00600097F5E3FAB9D0600097F5E4FAB5D07B
:1008DC00600097F5E5FAB1D0600097F5E6FAADD077
:1008EC00600097F5E8FAA9D0600097F5E9FAA5D071
:1008FC0001016751000AD8B457D76751010AD8B41F
:10090C0057D76751020AD8B457D76751030AD8B4DE
:10091C0057D76751040AD8B457D76751050AD8B4CA
:10092C0057D76751060AD8B457D76751070AD8B4B6
:10093C0057D76751080AD8B457D76751090AD8B4A2
:10094C0057D767510A0AD8B457D767510B0AD8B48E
:10095C0057D767510C0AD8B457D767510D0AD8B47A
:10096C0057D767510E0AD8B457D767510F0AD8B466
:10097C0057D76751100AD8B457D76751110AD8B452
:10098C0057D76751120AD8B457D76751130AD8B43E
:10099C0057D76751140AD8B457D76751150AD8B42A
:1009AC0057D76751160AD8B457D76751170AD8B416
:1009BC0057D76751180AD8B457D76751190AD8B402
:1009CC0057D767511A0AD8B457D767511B0AD8B4EE
:1009DC0057D767511C0AD8B457D767511D0AD8B4DA
:1009EC0057D767511E0AD8B457D767511F0AD8B4C6
:1009FC0057D76751200AD8B457D76751210AD8B4B2
:100A0C0057D76751220AD8B457D76751230AD8B49D
:100A1C0057D76751240AD8B457D76751250AD8B489
:100A2C0057D76751260AD8B457D76751270AD8B475
:100A3C0057D76751280AD8B457D70101685302E039
:100A4C00E6EC00F0A8D0010166B102D0C29001D052
:100A5C00C280F9D0010166B102D0C29201D0C2822B
:100A6C00F2D0010166B102D0C29401D0C284EBD0A5
:100A7C00010166B102D0C29601D0C286E4D0010158
:100A8C0066B102D0C29801D0C288DDD0010166B136
:100A9C0002D0C29A01D0C28AD6D0010166B102D06E
:100AAC00C29C01D0C28CCFD0010166B102D0C29ED3
:100ABC0001D0C28EC8D0010166B102D0C39001D062
:100ACC00C380C1D0010166B102D0C39201D0C382F0
:100ADC00BAD0010166B102D0C39401D0C384B3D0A3
:100AEC00010166B102D0C39601D0C386ACD001011E
:100AFC0066B102D0C39801D0C388A5D0010166B1FC
:100B0C0002D0C39A01D0C38A9ED0010166B102D033
:100B1C00C39C01D0C38C97D0010166B102D0C39E97
:100B2C0001D0C38E90D0010166B102D0C49001D027
:100B3C00C48089D0010166B102D0C49201D0C482B4
:100B4C0082D0010166B102D0C49401D0C4847BD0A0
:100B5C00010166B102D0C49601D0C48674D00101E3
:100B6C0066B102D0C49801D0C4886DD0010166B1C1
:100B7C0002D0C49A01D0C48A66D0010166B102D0F9
:100B8C00C49C01D0C48C5FD0010166B102D0C49E5C
:100B9C0001D0C48E58D001016551000AD8B453D786
:100BAC006551010AD8B456D76551020AD8B459D741
:100BBC006551030AD8B45CD76551040AD8B45FD721
:100BCC006551050AD8B462D76551060AD8B465D701
:100BDC006551070AD8B468D76551080AD8B46BD7E1
:100BEC006551090AD8B46ED765510A0AD8B471D7C1
:100BFC0065510B0AD8B474D765510C0AD8B477D7A1
:100C0C0065510D0AD8B47AD765510E0AD8B47DD780
:100C1C0065510F0A81E06551100A85E06551110A92
:100C2C0089E06551120A8DE06551130A91E0655116
:100C3C00140A95E06551150A99E06551160A9DE074
:0C0C4C006551170AA1E0FF0E006E1200B7
:100C58000B800BAE38EF06F0026A0AAEFF0E026E8A
:0C0C6800016E006E0A360232FF0E120010
:100C7400025006180E6E086A096A0B6A035007646C
:100C84002DEF07F006500A6E068E028E03500B6E8F
:100C94000750036E000E0B647DEF06F00B50075EE9
:100CA400D8B41EEF07F0070E0764ECEF06F0075EFA
:100CB40000C008F001C000F002C001F0026A074E53
:100CC4001EEF07F00764C1EF06F0075E00C008F0EE
:100CD40001C000F0016A074E1EEF07F007649FEFA2
:100CE40006F0075E00C008F0006A074E1EEF07F02A
:100CF400076486EF06F00AC002F005C001F004C0E4
:100D040000F0086A4AEF08F0030E076491EF06F05A
:100D1400075E08380F0B086E074E1EEF07F0D890D9
:100D24000832074E1EEF07F0D8900832074E1EEF28
:100D340007F0D89008321EEF07F0030E0764B0EFF7
:100D440006F0075E08380F0B086E0038F00B082613
:100D540000380F0B006E074E1EEF07F0D8900032DC
:100D64000832074E1EEF07F0D89000320832074EC3
:100D74001EEF07F0D890003208321EEF07F0030E82
:100D84000764D8EF06F0075E08380F0B086E0038CA
:100D9400F00B082600380F0B006E0138F00B00260C
:100DA40001380F0B016E074E1EEF07F0D890013289
:100DB40000320832074E1EEF07F0D890013200329D
:100DC4000832074E1EEF07F0D89001320032083285
:100DD4001EEF07F0030E076409EF07F0075E0838FB
:100DE4000F0B086E0038F00B082600380F0B006E4E
:100DF4000138F00B002601380F0B016E0238F00B9E
:100E0400012602380F0B026E074E1EEF07F0D89032
:100E14000232013200320832074E1EEF07F0D8903A
:100E24000232013200320832074E1EEF07F0D8902A
:100E34000232013200320832096A000E0EAE12EF9D
:100E440008F0081E001E011E021E082A00220122AC
:100E5400022212EF08F00750D8A433EF07F04AEF4C
:100E640008F0096A02C00AF0028E068E0750035C7D
:100E7400076ED8B405EF08F0070E0764D3EF07F048
:100E8400075E0450096E0550046E0650056E066A2E
:100E9400074E05EF08F0070E0764A8EF07F0075E9A
:100EA4000450096E0550046E056A074E05EF08F0FC
:100EB400070E076486EF07F0075E0450096E046AA4
:100EC400074E05EF08F0070E07646DEF07F00AC040
:100ED40002F04AEF08F0030E076478EF07F0075EAC
:100EE40009380F0B096E074E05EF08F0D890093248
:100EF400074E05EF08F0D8900932074E05EF08F0C9
:100F0400D890093205EF08F0030E076497EF07F055
:100F1400075E09380F0B096E0438F00B09260438F4
:100F24000F0B046E074E05EF08F0D8900432093217
:100F3400074E05EF08F0D89004320932074E05EF4A
:100F440008F0D8900432093205EF08F0030E076464
:100F5400BFEF07F0075E09380F0B096E0438F00B7A
:100F6400092604380F0B046E0538F00B04260538E7
:100F74000F0B056E074E05EF08F0D89005320432CA
:100F84000932074E05EF08F0D890053204320932D1
:100F9400074E05EF08F0D89005320432093205EF08
:100FA40008F0030E0764F0EF07F0075E09380F0B33
:100FB400096E0438F00B092604380F0B046E05384B
:100FC400F00B042605380F0B056E0638F00B0526CA
:100FD40006380F0B066E074E05EF08F0D890063260
:100FE400053204320932074E05EF08F0D890063274
:100FF400053204320932074E05EF08F0D890063264
:10100400053204320932086A000E0EAE12EF08F0FF
:10101400091E041E051E061E092A04220522062294
:1010240009500826045000220550012206500222CD
:101034000EBE29EF08F0D8A038EF08F002320132D2
:1010440000320832033E38EF08F044EF08F0D8B01D
:101054003EEF08F0000E081E001E011E021E082AA4
:101064000022012202220A7E3EEF08F0010E0C6EDD
:10107400FCEC00F04CEF08F0020E0C6EFCEC00F0FF
:101084004CEF08F0040E0C6EB0EC00F04CEF08F0DE
:06109400000E0C6E1200BC
:10109A00D250026ED29E0500FF6A0150FE6E0050C9
:0810AA00FD6E02BED28E1200A1
:1010B20003500718D8A46DEF08F002500618D8A400
:1010C2006DEF08F001500518D8A46DEF08F000503C
:0E10D2000418D8B4D8841200D894120012006A
:1010E000800E01016019006E800E000A005CD8B00D
:1010F00085D160510008016E01C060F1800E0118B9
:10110000006E800E6E0A005CD8A0CCD0640E046E17
:1011100060C100F0B8EC02F0120E0024056E000E63
:1011200000BEFF0E066E000E062205C000F006C0CF
:1011300001F0000E06BEFF0E026E036E0036009038
:101140000136023603360036009001360236033689
:101150007D0E0024F66E540E0120F76E000E022064
:10116000F86E09006F00D4FF61F109006F00D4FF31
:1011700062F109006F00D4FF63F109006F00D4FF32
:1011800064F1640E046E60C100F0B8EC02F008C0B7
:1011900000F00A0E046EB8EC02F0090E0024056E91
:1011A000000E00BEFF0E066E000E062205C000F007
:1011B00006C001F0000E06BEFF0E026E036E003682
:1011C00000900136023603360036009001360236B2
:1011D00003367D0E0024F66E540E0120F76E000ECD
:1011E0000220F86E09006F00D4FF00F009006F00C4
:1011F000D4FF01F009006F00D4FF02F009006F0076
:10120000D4FF03F061C104F062C105F063C106F0D0
:1012100064C107F0F5EC01F000C061F101C062F1BA
:1012200002C063F103C064F10A0E046E60C100F0F5
:10123000B8EC02F008C000F000C001F0000E00BEE3
:10124000FF0E026E036E046E013601900236033605
:101250000436013601900236033604367D0E012431
:10126000F66E540E0220F76E000E0320F86E090091
:101270006F00D4FF00F009006F00D4FF01F00900F7
:101280006F00D4FF02F009006F00D4FF03F061C1CA
:1012900004F062C105F063C106F064C107F0F5EC2B
:1012A00001F02BD2800E0A0A006E800E6019005CDD
:1012B00079E20A0E046E60C100F0B8EC02F0090E8B
:1012C0000024056E000E00BEFF0E066E000E062204
:1012D00005C000F006C001F0000E06BEFF0E026E53
:1012E000036E003600900136023603360036009059
:1012F0000136023603367D0E0024F66E540E0120B0
:10130000F76E000E0220F86E09006F00D4FF61F145
:1013100009006F00D4FF62F109006F00D4FF63F190
:1013200009006F00D4FF64F10A0E046E60C100F082
:10133000B8EC02F008C000F000C001F0000E00BEE2
:10134000FF0E026E036E046E013601900236033604
:101350000436013601900236033604367D0E012430
:10136000F66E540E0220F76E000E0320F86E090090
:101370006F00D4FF00F009006F00D4FF01F00900F6
:101380006F00D4FF02F009006F00D4FF03F061C1C9
:1013900004F062C105F063C106F064C107F0F5EC2A
:1013A00001F0ABD160C100F0000E60BFFF0E016E16
:1013B000026E036E003600900136023603360036A8
:1013C00000900136023603367D0E0024F66E540E70
:1013D0000120F76E000E0220F86E09006F00D4FFA6
:1013E00000F009006F00D4FF01F009006F00D4FF86
:1013F00002F009006F00D4FF03F07FD1800E601966
:10140000006E800E6E0A005CD8A0CCD0640E046E14
:1014100060C100F0B8EC02F0120E0024056E000E60
:1014200000BEFF0E066E000E062205C000F006C0CC
:1014300001F0000E06BEFF0E026E036E0036009035
:101440000136023603360036009001360236033686
:10145000B10E0024F66E540E0120F76E000E02202D
:10146000F86E09006F00D4FF61F109006F00D4FF2E
:1014700062F109006F00D4FF63F109006F00D4FF2F
:1014800064F1640E046E60C100F0B8EC02F008C0B4
:1014900000F00A0E046EB8EC02F0090E0024056E8E
:1014A000000E00BEFF0E066E000E062205C000F004
:1014B00006C001F0000E06BEFF0E026E036E00367F
:1014C00000900136023603360036009001360236AF
:1014D0000336B10E0024F66E540E0120F76E000E96
:1014E0000220F86E09006F00D4FF00F009006F00C1
:1014F000D4FF01F009006F00D4FF02F009006F0073
:10150000D4FF03F061C104F062C105F063C106F0CD
:1015100064C107F0F5EC01F000C061F101C062F1B7
:1015200002C063F103C064F10A0E046E60C100F0F2
:10153000B8EC02F008C000F000C001F0000E00BEE0
:10154000FF0E026E036E046E013601900236033602
:10155000043601360190023603360436B10E0124FA
:10156000F66E540E0220F76E000E0320F86E09008E
:101570006F00D4FF00F009006F00D4FF01F00900F4
:101580006F00D4FF02F009006F00D4FF03F061C1C7
:1015900004F062C105F063C106F064C107F0F5EC28
:1015A00001F0ABD0800E0A0A006E800E6019005C5C
:1015B00079E20A0E046E60C100F0B8EC02F0090E88
:1015C0000024056E000E00BEFF0E066E000E062201
:1015D00005C000F006C001F0000E06BEFF0E026E50
:1015E000036E003600900136023603360036009056
:1015F000013602360336B10E0024F66E540E012079
:10160000F76E000E0220F86E09006F00D4FF61F142
:1016100009006F00D4FF62F109006F00D4FF63F18D
:1016200009006F00D4FF64F10A0E046E60C100F07F
:10163000B8EC02F008C000F000C001F0000E00BEDF
:10164000FF0E026E036E046E013601900236033601
:10165000043601360190023603360436B10E0124F9
:10166000F66E540E0220F76E000E0320F86E09008D
:101670006F00D4FF00F009006F00D4FF01F00900F3
:101680006F00D4FF02F009006F00D4FF03F061C1C6
:1016900004F062C105F063C106F064C107F0F5EC27
:1016A00001F02BD060C100F0000E60BFFF0E016E94
:1016B000026E036E003600900136023603360036A5
:1016C0000090013602360336B10E0024F66E540E39
:1016D0000120F76E000E0220F86E09006F00D4FFA3
:1016E00000F009006F00D4FF01F009006F00D4FF83
:0C16F00002F009006F00D4FF03F01200AC
:1016FC000450000A08E10550000A05E1FF0E006ED7
:10170C007F0E016E58D00D6A096A086A01500010EC
:10171C00D8B4000C015005180A6E0ABE0D1E0B6AD7
:10172C0005AE05D0041E051E042AD8B4052A01AE48
:10173C0005D0001E011E002AD8B4012A0150051044
:10174C000A6E0ABE10D08CEC02F00BB020D00DAE9D
:10175C00000C001E011E002AD8B4012A081E091E06
:10176C00082AD8B4092A000C05AE0DD001BE07D04A
:10177C000150096E0050086E016A006AE8D7016AD0
:10178C00006A002A000C011E001E0B2ADDD7082A55
:10179C00D8B4092A0450085CD8A4D9D70550095CE0
:1017AC00D8A4D5D7096A086A002AD8B4012A01AE90
:0817BC00CED70000FF0C120063
:1017C40001016051390806E3300E605D03E3010E48
:0817D400006E01D0006A120052
:1017DC00600067F4E1FF60006BF4E2FF600083F5EA
:0E17EC00E6FF17C100F018C101F051DC120039
:1017FA000A6A0350D8A40A800750D8A40A820A5059
:10180A00D8B460EF0CF0030AD8B419EF0CF00AB0A0
:10181A0014EF0CF006AE5EEF0CF05CEF0CF002AECB
:10182A005CEF0CF05EEF0CF00250800B0A6E029E29
:10183A000650800B069E0A18D8B42AEF0CF00A50FC
:10184A00D8B45CEF0CF05EEF0CF00750035CD8B430
:10185A0034EF0CF0D8A050EF0CF056EF0CF0065015
:10186A00025CD8B43EEF0CF0D8A050EF0CF056EF63
:10187A000CF00550015CD8B448EF0CF0D8A050EF3A
:10188A000CF056EF0CF00450005CD8B460EF0CF08A
:10189A00D8B056EF0CF00A52D8B45EEF0CF05CEFF9
:1018AA000CF00A52D8B45CEF0CF05EEF0CF0D88062
:0E18BA001200D8901200D880D88412001200BC
:1018C8000B6A0A6A096A005004026F00D0FF09F027
:1018D8006F00CCFF08F0015005026F00D0FF0BF03D
:1018E8006F00CCFF0AF000500502F3500926F450AF
:1018F8000A22E86A0B2201500402F3500926F45028
:101908000A22E86A0B2208C000F009C001F00AC0E8
:0819180002F00BC003F0120005
:101920000450000A12E10550000A0FE10650000AB7
:101930000CE10750000A09E1FF0E006EFF0E016E78
:101940007F0E026EFF0E036EA8D0086A096A075068
:10195000D8B43BEF0DF00350D8B440EF0DF0025077
:1019600006180A6E028E068E0E6A02C008F001C0CA
:101970000CF000C00DF004500D5E0550D8A0053CE1
:101980000C5E0650D8A0063C085E086A0C6A0D6A18
:10199000D8A0D2EF0CF0D8900232013200320832D7
:1019A000010E0E6E0750035ED8A0DFEF0CF07E0E26
:1019B0000E240326D8B045EF0DF0E5EF0CF07E0EB7
:1019C0000E240326D8A04AEF0DF0180E0B6E0D362C
:1019D0000C3608360036013602360E360450005EEC
:1019E0000550D8A0053C015E0650D8A0063C025E1A
:1019F00006340E120EA000EF0DF00D800BEF0DF06F
:101A0000045000260550D8B0053C01260650D8B039
:101A1000062802260D900B2EE7EF0CF031EF0DF0AB
:101A2000D8900036013602360E360450005E05505E
:101A3000D8A0053C015E0650D8A0063C025E0634E4
:101A40000E10010B0D26D8B00C2AD8B4082AD8A441
:101A500031EF0DF008320C320D32032AD8B445EFC5
:101A60000DF00AAE089E0850026E0C50016E0D502B
:101A7000006E4DEF0DF0010E88EC02F04DEF0DF011
:101A8000020EC9EC00F04DEF0DF0040EB0EC00F0CA
:0C1A90004DEF0DF0080ED9EC00F0120034
:101A9C006E0E0101605DD8A0D6D0640E046E60C1DC
:101AAC0000F007EC03F0120E0024056E066A000E1F
:101ABC00062205C000F006C001F0000E06BEFF0EA7
:101ACC00026E036E00360090013602360336003685
:101ADC0000900136023603367D0E0024F66E540E4D
:101AEC000120F76E000E0220F86E09006F00D4FF83
:101AFC0000F009006F00D4FF01F009006F00D4FF63
:101B0C0002F009006F00D4FF03F0000E046E000E0B
:101B1C00056E000E066E7E0E076EF5EC01F000C031
:101B2C0061F101C062F102C063F103C064F1640EA3
:101B3C00046E60C100F007EC03F008C000F00A0E60
:101B4C00046E07EC03F0090E0024056E066A000E05
:101B5C00062205C000F006C001F0000E06BEFF0E06
:101B6C00026E036E003600900136023603360036E4
:101B7C0000900136023603367D0E0024F66E540EAC
:101B8C000120F76E000E0220F86E09006F00D4FFE2
:101B9C0000F009006F00D4FF01F009006F00D4FFC2
:101BAC0002F009006F00D4FF03F061C104F062C1C0
:101BBC0005F063C106F064C107F0F5EC01F000C05C
:101BCC0061F101C062F102C063F103C064F10A0E5D
:101BDC00046E60C100F007EC03F008C000F000C018
:101BEC0001F0000E026E036E046E01360190023697
:101BFC0003360436013601900236033604367D0E68
:101C0C000124F66E540E0220F76E000E0320F86EBF
:101C1C0009006F00D4FF00F009006F00D4FF01F041
:101C2C0009006F00D4FF02F009006F00D4FF03F02D
:101C3C0061C104F062C105F063C106F064C107F034
:101C4C00F5EC01F0BDD060510A08D8B086D00A0E70
:101C5C00046E60C100F007EC03F0090E0024056E61
:101C6C00066A000E062205C000F006C001F0000E48
:101C7C0006BEFF0E026E036E003600900136023671
:101C8C000336003600900136023603367D0E0024F2
:101C9C00F66E540E0120F76E000E0220F86E09004D
:101CAC006F00D4FF00F009006F00D4FF01F00900B1
:101CBC006F00D4FF02F009006F00D4FF03F0000E98
:101CCC00046E000E056E000E066E7E0E076EF5ECB1
:101CDC0001F000C061F101C062F102C063F103C008
:101CEC0064F10A0E046E60C100F007EC03F008C04A
:101CFC0000F000C001F0000E026E036E046E01369F
:101D0C000190023603360436013601900236033652
:101D1C0004367D0E0124F66E540E0220F76E000E72
:101D2C000320F86E09006F00D4FF00F009006F006B
:101D3C00D4FF01F009006F00D4FF02F009006F001E
:101D4C00D4FF03F061C104F062C105F063C106F079
:101D5C0064C107F0F5EC01F033D060C100F0000E67
:101D6C00016E026E036E00360090013602360336A9
:101D7C00003600900136023603367D0E0024F66ED6
:101D8C00540E0120F76E000E0220F86E09006F0051
:101D9C00D4FF00F009006F00D4FF01F009006F00C0
:101DAC00D4FF02F009006F00D4FF03F0000E046EA4
:101DBC00000E056E000E066E7E0E076EF5EC01F041
:021DCC00120003
:101DCE000B6A0C6A086A0350D8B46BEF0FF002C0AE
:101DDE000AF0028E9E0E035E03AE5BEF0FF0036CF5
:101DEE00080E035CD8A028EF0FF0036E083600C073
:101DFE0008F001C000F002C001F0026A080E035C98
:101E0E00D8A028EF0FF0036E083600C008F001C00E
:101E1E0000F0016A080E035CD8A028EF0FF0036EE5
:101E2E00083600C008F0006A080E035CD8A028EF40
:101E3E000FF0036E0836086A0350D8A4D89034EF1A
:101E4E000FF00350D8B434EF0FF0D89002320132B5
:101E5E0000320832032E2CEF0FF00BBC08A045EF1A
:101E6E000FF0D8A045EF0FF0082AD8B4002AD8B446
:101E7E00012AD8B4022A02BE6FEF0FF00AAE6BEF42
:101E8E000FF0021E011E001E081E082AD8B4002ADA
:101E9E00D8B4012AD8B4022A6BEF0FF0026A016A95
:101EAE00006A086A6BEF0FF00B800BAE76EF0FF047
:101EBE00026A0AAE76EF0FF0026E016E006E086EC9
:101ECE000A36023276EF0FF00C6A000E77EF0FF043
:101EDE00010E0C6E000E2CEC06F077EF0FF0FF0EDD
:101EEE000250036E0150026E0050016E0850006EDB
:021EFE001200D0
:0A1F0000490E0D6E0D2EFED71200E3
:101F0A000B6A0A6A096A086A0E6A033408360450B8
:101F1A00085E0550D8A0053C095E0650D8A0063CCC
:101F2A000A5E0750D8A0073C0B5EE86AD8A0010EEB
:101F3A000E5E0336070E0C6E0334083609360A366F
:101F4A000B360E36045003A012D0085E0550D8A0F6
:101F5A00053C095E0650D8A0063C0A5E0750D8A088
:101F6A00073C0B5EE86AD8A0010E0E5E11D0082667
:101F7A000550D8B0053C09260650D8B0063C0A26BA
:101F8A000750D8B0073C0B26E86AD8B0010E0E26D7
:101F9A0003360C2ED1D70234083609360A360B36E8
:101FAA000E36045003A012D0085E0550D8A0053C96
:101FBA00095E0650D8A0063C0A5E0750D8A0073C26
:101FCA000B5EE86AD8A0010E0E5E11D008260550F5
:101FDA00D8B0053C09260650D8B0063C0A26075058
:101FEA00D8B0073C0B26E86AD8B0010E0E26023696
:101FFA00070E0C6E0234083609360A360B360E36D0
:10200A00045002A012D0085E0550D8A0053C095E13
:10201A000650D8A0063C0A5E0750D8A0073C0B5EC3
:10202A00E86AD8A0010E0E5E11D008260550D8B075
:10203A00053C09260650D8B0063C0A260750D8B0F7
:10204A00073C0B26E86AD8B0010E0E2602360C2E83
:10205A00D1D70134083609360A360B360E36045003
:10206A0002A012D0085E0550D8A0053C095E0650B1
:10207A00D8A0063C0A5E0750D8A0073C0B5EE86A67
:10208A00D8A0010E0E5E11D008260550D8B0053C26
:10209A0009260650D8B0063C0A260750D8B0073C95
:1020AA000B26E86AD8B0010E0E260136070E0C6E12
:1020BA000134083609360A360B360E36045001A0AA
:1020CA0012D0085E0550D8A0053C095E0650D8A07B
:1020DA00063C0A5E0750D8A0073C0B5EE86AD8A007
:1020EA00010E0E5E11D008260550D8B0053C09260F
:1020FA000650D8B0063C0A260750D8B0073C0B2633
:10210A00E86AD8B0010E0E2601360C2ED1D700345B
:10211A00083609360A360B360E36045001A012D09C
:10212A00085E0550D8A0053C095E0650D8A0063CBA
:10213A000A5E0750D8A0073C0B5EE86AD8A0010ED9
:10214A000E5E11D008260550D8B0053C0926065067
:10215A00D8B0063C0A260750D8B0073C0B26E86AD6
:10216A00D8B0010E0E260036070E0C6E0034083663
:10217A0009360A360B360E36045000A012D0085E15
:10218A000550D8A0053C095E0650D8A0063C0A5E58
:10219A000750D8A0073C0B5EE86AD8A0010E0E5E75
:1021AA0011D008260550D8B0053C09260650D8B0EB
:1021BA00063C0A260750D8B0073C0B26E86AD8B076
:1021CA00010E0E2600360C2ED1D700B00ED00450C8
:1021DA0008260550D8B0053C09260650D8B0063C5A
:0C21EA000A260750D8B0073C0B26120054
:0821F600067E3AEC06F012002F
:1021FE0060C165F161C166F162C167F1010E010155
:08220E00686F16EC03F01200EA
:102216000B6A0C6A0A6A086A0350D8B493EF11F085
:10222600028E9E0E035E03BE1EEF11F0D8B41EEFA3
:1022360011F083EF11F0036C080E035CD8A050EF89
:1022460011F0036E083600C008F001C000F002C0AD
:1022560001F0026A080E035CD8A050EF11F0036E7D
:10226600083600C008F001C000F0016A080E035CE1
:10227600D8A050EF11F0036E083600C008F0006ACF
:10228600080E035CD8A050EF11F0036E0836086AFA
:102296000350D8A4D8905CEF11F00350D8B45CEF8B
:1022A60011F0D8900232013200320832032E54EF78
:1022B60011F00BBC08A06DEF11F0D8A06DEF11F076
:1022C600082AD8B4002AD8B4012AD8B4022A02BEF1
:1022D60097EF11F00AAE93EF11F0021E011E001ED9
:1022E600081E082AD8B4002AD8B4012AD8B4022A6B
:1022F60093EF11F0026A016A006A086A93EF11F01F
:102306000B800BAE9DEF11F0026A0AAE9DEF11F045
:10231600026E016E006E086E0A3602329DEF11F0F3
:10232600000E0C6A9EEF11F0010E0C6E2CEC06F0FE
:102336009EEF11F0FF0E0250036E0150026E005028
:08234600016E0850006E120048
:10234E000050086E0150006E0250016E0350026E76
:10235E00036A0B6A0C6A9E0E036E0A6A020E0C6EFC
:06236E00FCEC00F012007F
:102374000101586B596B4C6B4D6B3AC100F03BC17A
:1023840001F03CC102F0010E3A27000E3B233C232E
:10239400600003F0F6FF600007F0F7FF60000BF049
:1023A400F8FF09006F00D4FF00F000C049F10052AB
:1023B400D8B439EF23F04951250A0EE06000E3F464
:1023C400E1FF6000E7F4E2FF600027F5E6FF384B29
:1023D400392B584B592BD1D74A6B4B6B4C6B4D6BEC
:1023E40023D04C87010E3A27000E3B233C236DD0AB
:1023F4004C81010E3A27000E3B233C2366D04C83CC
:10240400010E3A27000E3B233C235FD04D87010E7B
:102414003A27000E3B233C2358D04C85010E3A2723
:10242400000E3B233C2351D06000EBF4F6FF600028
:10243400EFF4F7FF6000F3F4F8FF09006F00D4FF36
:1024440001F001502D0ACDE06000EBF4F6FF6000CE
:10245400EFF4F7FF6000F3F4F8FF09006F00D4FF16
:1024640001F00150200AC4E06000EBF4F6FF6000C4
:10247400EFF4F7FF6000F3F4F8FF09006F00D4FFF6
:1024840001F001502B0ABBE06000EBF4F6FF6000A2
:10249400EFF4F7FF6000F3F4F8FF09006F00D4FFD6
:1024A40001F00150230AB2E06000EBF4F6FF600093
:1024B400EFF4F7FF6000F3F4F8FF09006F00D4FFB6
:1024C40001F00150300AA9E001D08AD74CA301D011
:1024D4004C914CA701D04C956000EBF4F6FF6000E2
:1024E400EFF4F7FF6000F3F4F8FF09006F00D4FF86
:1024F40000F0000E016E00C060F1E2EC0BF000523F
:102504003EE04A6B4B6B4AC100F04BC101F00A0E2E
:10251400046E000E056E64EC0CF06000EBF4F6FF44
:102524006000EFF4F7FF6000F3F4F8FF09006F00B8
:10253400D4FF02F0025000244A6F000E01204B6FBA
:10254400300E4A5F000E4B5B010E3A27000E3B2310
:102554003C236000EBF4F6FF6000EFF4F7FF60004B
:10256400F3F4F8FF09006F00D4FF00F0000E016ED1
:1025740000C060F1E2EC0BF00052C5E145D0600010
:10258400EBF4F6FF6000EFF4F7FF6000F3F4F8FFFC
:1025940009006F00D4FF01F001502A0A35E1600000
:1025A400F7F4E9FF6000FBF4EAFF6F00B8FF00F006
:1025B4006F00B8FF01F0600003F0E9FF600007F06E
:1025C400EAFF6F00B8FF4AF16F00B8FF4BF16000FB
:1025D400F7F4E9FF6000FBF4EAFF020EEE24006E5C
:1025E400000EEE20016E6000F7F4E1FF6000FBF4E2
:1025F400E2FF600003F0E6FF600007F0E6FF010E73
:102604003A27000E3B233C236000EBF4F6FF600006
:10261400EFF4F7FF6000F3F4F8FF09006F00D4FF54
:1026240001F001502E0AD8A48AD0010E3A27000ED8
:102634003B233C236000EBF4F6FF6000EFF4F7FF6C
:102644006000F3F4F8FF09006F00D4FF01F00150BB
:102654002A0A36E16000F7F4E9FF6000FBF4EAFFC0
:102664006F00B8FF00F06F00B8FF01F0600003F0E6
:10267400E9FF600007F0EAFF6F00B8FF47F16F0061
:10268400B8FF48F16000F7F4E9FF6000FBF4EAFFEB
:10269400020EEE24006E000EEE20016E6000F7F4D0
:1026A400E1FF6000FBF4E2FF600003F0E6FF60007E
:1026B40007F0E6FF010E3A27000E3B233C233ED0F1
:1026C400476B486B6000EBF4F6FF6000EFF4F7FF34
:1026D4006000F3F4F8FF09006F00D4FF00F0000E6F
:1026E400016E00C060F1E2EC0BF0005227E047C13C
:1026F40000F048C101F00A0E046E000E056E64EC91
:102704000CF06000EBF4F6FF6000EFF4F7FF6000FC
:10271400F3F4F8FF09006F00D4FF02F00250002424
:10272400476F000E0120486F300E475F000E485B74
:10273400010E3A27000E3B233C23C4D703D0476B3A
:10274400486B4D893AC100F03BC101F03CC102F035
:10275400010E3A27000E3B233C23600003F0F6FFF2
:10276400600007F0F7FF60000BF0F8FF09006F004E
:10277400D4FF49F11DD158C100F059C101F03DEF1A
:1027840023F04C89DFD74D8552D14C8B4D814FD1ED
:102794004D834DD14C8D4BD14AD14C8B4C8F47D16D
:1027A4006000F7F4E9FF6000FBF4EAFF6F00B8FF94
:1027B40000F06F00B8FF01F0600003F0E9FF600073
:1027C40007F0EAFF6F00B8FF54F16F00B8FF55F14E
:1027D4006000F7F4E9FF6000FBF4EAFF020EEE2468
:1027E400006E000EEE20016E6000F7F4E1FF600061
:1027F400FBF4E2FF600003F0E6FF600007F0E6FF91
:10280400000E551902E1000E541904E1240E546F10
:10281400000E556F566B576B56515425E96E575140
:102824005521EA6EEE520BE0010E5625006E000EA5
:102834005721016E00C056F101C057F1EDD7475141
:1028440048110AE05751485D02E15651475D04E2E0
:1028540047C156F148C157F14B51575D02E14A5106
:10286400565D05E256514A5F57514B5B02D04A6BA5
:102874004B6B4CB718D04AC100F04BC101F0010EAC
:102884004A5F000E4B5B005001100DE06000E3F462
:10289400E1FF6000E7F4E2FF200EE66E384B392BCF
:1028A400584B592BE8D756C102F057C103F0010E1B
:1028B400565D006E000E5759016E00C056F101C0FE
:1028C40057F1025003101EE0600053F5E9FF600069
:1028D40057F5EAFF6000E3F4E1FF6000E7F4E2FF8C
:1028E4006F00BBFFE6FF384B392B010E5425006EF9
:1028F400000E5521016E00C054F101C055F1584B32
:10290400592BD1D74CA718D04AC100F04BC101F0C4
:10291400010E4A5F000E4B5B005001100DE0600099
:10292400E3F4E1FF6000E7F4E2FF200EE66E384BCB
:10293400392B584B592BE8D720D56000F7F4E9FF21
:102944006000FBF4EAFF6F00B8FF00F06F00B8FF0F
:1029540001F0600003F0E9FF600007F0EAFF6F0098
:10296400B8FF49F16000F7F4E9FF6000FBF4EAFF07
:10297400020EEE24006E000EEE20016E6000F7F4ED
:10298400E1FF6000FBF4E2FF600003F0E6FF60009B
:1029940007F0E6FF490E546F010E556F010E566F96
:1029A400000E576F4CD7C00E4C13000E4D133FD082
:1029B4004951000AD8B4DFD649516C0AD8B4E1D6DB
:1029C40049514C0AD8B4DDD64951660AD8B4DBD68D
:1029D4004951450AD8B4D9D64951650AD8B4D6D68E
:1029E4004951670AD8B4D4D649516F0AD8B4D2D65B
:1029F4004951640AD8B4D0D64951690AD8B4CCD65E
:102A04004951700AD8B4C9D64951580AD8B4C5D660
:102A14004951780AD8B4C2D64951730AD8B4C0D639
:102A24004951630A8AE04951750ABDE0B3D7000EE3
:102A34004C15006E4D51070B016E00500110D8B4B7
:102A440064EF1EF04DA904D0060E476F000E486FC8
:102A54006000F7F4E9FF6000FBF4EAFF6F00B8FFE1
:102A640000F06F00B8FF01F0600003F0E9FF6000C0
:102A740007F0EAFF6F00B8FF4EF16F00B8FF4FF1A7
:102A84006F00B8FF50F16F00B8FF51F16000F7F428
:102A9400E9FF6000FBF4EAFF040EEE24006E000E72
:102AA400EE20016E6000F7F4E1FF6000FBF4E2FF4A
:102AB400600003F0E6FF600007F0E6FF046A056AC1
:102AC400066A076A4EC100F04FC101F050C102F01E
:102AD40051C103F0FDEC0BF0010ED8B0000E006EF6
:102AE400005205E0507F030E4C13000E4D13526B41
:102AF400536B4EC100F04FC101F050C102F051C1FF
:102B040003F0046A056A066A076A59EC08F0000EC5
:102B1400D8A4010E006E0052D8B48AD051C100F07E
:102B2400016A026A036AFF0E0016000E01167E0E89
:102B3400005E000E015A00C052F101C053F1010EB3
:102B4400005E000E015A00C052F101C053F1030EA1
:102B5400046E000E056E64EC0CF000C052F101C06E
:102B640053F10A0E046E000E056E7EEC0BF000C0ED
:102B740052F101C053F1800E0118026E800E025C06
:102B840002E1000E005C05E2010E0101525F000E3D
:102B9400535B010152510008606F70EC08F04EC1A4
:102BA40004F04FC105F050C106F051C107F0F5EC37
:102BB40001F000C054F101C055F102C056F103C048
:102BC40057F1000E046E000E056E000E066E7F0EA9
:102BD400076E54C100F055C101F056C102F057C14F
:102BE40003F0FDEC0BF0010ED8B0000E006E0052A5
:102BF40005E0010E525F000E535B1AD0000E046E06
:102C0400000E056E200E066E820E076E54C100F093
:102C140055C101F056C102F057C103F0FDEC0BF0B1
:102C2400000ED8B0010E006E005202E0524B532B3E
:102C3400800E006E800E5319005C02E152510008B0
:102C440003E3010E496F02D052C149F14DB119D0CD
:102C54004DA315D0800E5319006E7F0E005C02E167
:102C6400FC0E525D0BE3800E5319006E800E481962
:102C7400005C02E14751525D01E201D002D06AEFEB
:102C84001AF04751481106E04DA304D0010E475FE6
:102C9400000E485B4851000802E14751080803E26E
:102CA400080E496F02D047C149F14EC100F04FC12F
:102CB40001F050C102F051C103F0046A056A066ACA
:102CC400076A59EC08F0000ED8A4010E006E0052F9
:102CD400D8B453D152C160F170EC08F000C004F0D4
:102CE40001C005F002C006F003C007F04EC100F0B9
:102CF4004FC101F050C102F051C103F090EC0CF04F
:102D040000C04EF101C04FF102C050F103C051F1B7
:102D1400010149510008606F70EC08F000C004F034
:102D240001C005F002C006F003C007F04EC100F078
:102D34004FC101F050C102F051C103F090EC0CF00E
:102D440000C05AF101C05BF102C05CF103C05DF147
:102D54005AC14EF15BC14FF15CC150F15DC151F1FB
:102D64005AC100F05BC101F05CC102F05DC103F027
:102D74000BEC11F0A7EC11F000C004F001C005F059
:102D840002C006F003C007F05AC100F05BC101F0B5
:102D94005CC102F05DC103F0FBEC10F0000E046EA8
:102DA400000E056E000E066E7E0E076EFDEC0BF037
:102DB400000ED8B0010E006E00521AE04EC100F0B1
:102DC4004FC101F050C102F051C103F0000E046E76
:102DD400000E056E000E066E7E0E076E3AEC06F0CF
:102DE40000C04EF101C04FF102C050F103C051F1D7
:102DF4004EC100F04FC101F050C102F051C103F0C7
:102E04000BEC11F001014951010F096E0A6A000E21
:102E14000A2209C004F00AC005F0000E0ABEFF0E23
:102E2400066E076E043604900536063607360436F9
:102E34000490053606360736F70E0424F66E550E52
:102E44000520F76E000E0620F86E09006F00D4FF0F
:102E540005F009006F00D4FF06F009006F00D4FFED
:102E640007F009006F00D4FF08F00850035C08E184
:102E74000750025C05E10650015C02E10550005C6C
:102E84001EE301014EC100F04FC101F050C102F038
:102E940051C103F0CD0E046ECC0E056E4C0E066EC1
:102EA4007B0E076EF5EC01F000C04EF101C04FF14E
:102EB40002C050F103C051F1524B532B5ED04EC1AE
:102EC40000F04FC101F050C102F051C103F00BEC0E
:102ED40011F049C104F0000E056E066E076E04364B
:102EE4000490053606360736043604900536063651
:102EF4000736F70E0424F66E550E0520F76E000E05
:102F04000620F86E09006F00D4FF05F009006F0079
:102F1400D4FF06F009006F00D4FF07F009006F002A
:102F2400D4FF08F00850035C08E10750025C05E197
:102F34000650015C02E10550005C1FE201014EC134
:102F440000F04FC101F050C102F051C103F0000E76
:102F5400046E000E056E200E066E820E076EF5ECF2
:102F640001F000C04EF101C04FF102C050F103C0A6
:102F740051F1010E525F000E535B01014DA393D03A
:102F84004DB791D0800E000A006E800E4819005C87
:102F940002E147510A0804E20A0E476F000E486F27
:102FA4004EC100F04FC101F050C102F051C103F015
:102FB4000BEC11F000C054F101C055F102C056F100
:102FC40003C057F1545155115611571142E00A0EDE
:102FD400046E000E056E066E076E54C100F055C1F6
:102FE40001F056C102F057C103F085EC0FF008C0A0
:102FF40000F009C001F00AC002F00BC003F0000E9B
:10300400046E031808E10450021805E10450011885
:1030140002E10050000A1DE1010E475F000E485B0B
:103024000A0E046E000E056E066E076E54C100F0A3
:1030340055C101F056C102F057C103F085EC0FF001
:1030440000C054F101C055F102C056F103C057F15C
:10305400B9D7800E4819006E800E005C02E1495118
:10306400475D21E24751495D606F70EC08F000C094
:1030740004F001C005F002C006F003C007F04EC121
:1030840000F04FC101F050C102F051C103F090ECC7
:103094000CF000C04EF101C04FF102C050F103C06A
:1030A40051F147C149F1050E01014725006E000E9B
:1030B4004821016E00504A5F01504B5B4751481153
:1030C40003E14DB701D004D0010E4A5F000E4B5B03
:1030D400030E4C15006E4DC101F0000E0116005098
:1030E400011004E0010E4A5F000E4B5B4CA540D07A
:1030F4004CA315D04CA103D02D0E3F6F02D02B0E44
:103104003F6F6000E3F4E1FF6000E7F4E2FF60007A
:10311400FFF4E6FF384B392B584B592B0ED04CA1FA
:103124000CD06000E3F4E1FF6000E7F4E2FF200E5E
:10313400E66E384B392B584B592B800E006E800E9F
:103144004B19005C02E14A51000811E26000E3F40B
:10315400E1FF6000E7F4E2FF300EE66E384B392BF6
:10316400584B592B010E4A5F000E4B5BE6D741D0FA
:103174004CB71AD0800E006E800E4B19005C02E131
:103184004A51000811E26000E3F4E1FF6000E7F453
:10319400E2FF200EE66E384B392B584B592B010EAB
:1031A4004A5F000E4B5BE6D74CA315D04CA103D06D
:1031B4002D0E406F02D02B0E406F6000E3F4E1FF50
:1031C4006000E7F4E2FF600003F5E6FF384B392BBB
:1031D400584B592B0ED04CA10CD06000E3F4E1FF06
:1031E4006000E7F4E2FF200EE66E384B392B584BB3
:1031F400592B4EC100F04FC101F050C102F051C132
:1032040003F00BEC11F000C054F101C055F102C001
:1032140056F103C057F149C100F0000E016E026E71
:10322400036E0036009001360236033600360090F5
:10323400013602360336F70E0024F66E550E0120D1
:10324400F76E000E0220F86E09006F00D4FF04F040
:1032540009006F00D4FF05F009006F00D4FF06F0E9
:1032640009006F00D4FF07F054C100F055C101F00C
:1032740056C102F057C103F085EC0FF0300E002662
:103284006000E3F4E1FF6000E7F4E2FF600003F0B4
:10329400E6FF384B392B584B592B4751481103E162
:1032A4004DB701D07AD06000E3F4E1FF6000E7F4A9
:1032B400E2FF2E0EE66E384B392B584B592B4951F1
:1032C400475F000E485B495354E0490749C100F089
:1032D400000E016E026E036E003600900136023657
:1032E400033600360090013602360336F70E00240A
:1032F400F66E550E0120F76E000E0220F86E0900DE
:103304006F00D4FF04F009006F00D4FF05F009003A
:103314006F00D4FF06F009006F00D4FF07F054C11A
:1033240000F055C101F056C102F057C103F085EC1D
:103334000FF00A0E046E000E056E066E076E85EC25
:103344000FF008C000F009C001F00AC002F00BC081
:1033540003F0300E00266000E3F4E1FF6000E7F4C0
:10336400E2FF600003F0E6FF384B392B584B592B32
:10337400AAD74751481111E06000E3F4E1FF60006F
:10338400E7F4E2FF300EE66E384B392B584B592BDD
:10339400010E475F000E485BECD74CAB0DD06000CC
:1033A400E3F4E1FF6000E7F4E2FF450EE66E384B1C
:1033B400392B584B592B0CD06000E3F4E1FF60002B
:1033C400E7F4E2FF650EE66E384B392B584B592B68
:1033D400800E5319006E800E005C02E1000E525DF7
:1033E40013E252510008526F5351000E53576000BC
:1033F400E3F4E1FF6000E7F4E2FF2D0EE66E384BE4
:10340400392B584B592B0CD06000E3F4E1FF6000DA
:10341400E7F4E2FF2B0EE66E384B392B584B592B51
:103424000A0E046E000E056E52C100F053C101F085
:103434007EEC0BF0300E00266000E3F4E1FF600048
:10344400E7F4E2FF600003F0E6FF0101384B392B9B
:10345400584B592B0A0E046E000E056E52C100F033
:1034640053C101F07EEC0BF008C000F009C001F07C
:10347400300E00266000E3F4E1FF6000E7F4E2FFB1
:10348400600003F0E6FF0101384B392B584B592BF0
:103494004CA71CD0800E006E800E4B19005C02E11C
:1034A4004A51000813E26000E3F4E1FF6000E7F42E
:1034B400E2FF200EE66E384B392B584B592B010E88
:1034C4004A5F000E4B5B4A514B11EDE1BFEF11F027
:1034D4004DA3F7D0800E5319006E800E005C02E1FC
:1034E400000E525D0AE2010E525D006E000E535949
:1034F400016E0050475F0150485B4EC100F04FC160
:1035040001F050C102F051C103F00BEC11F000C006
:1035140054F101C055F102C056F103C057F1010E38
:10352400496F49510A0A38E049C100F0000E016EA2
:10353400026E036E00360090013602360336003602
:103544000090013602360336F70E0024F66E550E4F
:103554000120F76E000E0220F86E09006F00D4FF00
:1035640001F009006F00D4FF02F009006F00D4FFDE
:1035740003F009006F00D4FF04F00450575D08E124
:103584000350565D05E10250555D02E10150545D62
:1035940001E202D0492BC5D74951475D5E6F000E49
:1035A40048595F6F5EC147F15FC148F154C100F0F3
:1035B40055C101F056C102F057C103F0A7EC11F058
:1035C40000C004F001C005F002C006F003C007F01B
:1035D4004EC100F04FC101F050C102F051C103F0DF
:1035E400FBEC10F000C05AF101C05BF102C05CF1C9
:1035F40003C05DF15EC160F170EC08F05AC104F0E3
:103604005BC105F05CC106F05DC107F0F5EC01F0AB
:10361400000E046E000E056E000E066E7E0E076E22
:103624003AEC06F00BEC11F000C054F101C055F176
:1036340002C056F103C057F14751481142E00A0E47
:10364400046E000E056E066E076E54C100F055C17F
:1036540001F056C102F057C103F085EC0FF008C029
:1036640000F009C001F00AC002F00BC003F0000E24
:10367400046E031808E10450021805E1045001180F
:1036840002E10050000A1DE10A0E046E000E056EF0
:10369400066E076E54C100F055C101F056C102F028
:1036A40057C103F085EC0FF000C054F101C055F18F
:1036B40002C056F103C057F1010E475F000E485B8C
:1036C400BBD7800E006E800E4819005C02E14751A2
:1036D4000C0816E347C160F14EEC0DF04EC104F046
:1036E4004FC105F050C106F051C107F03AEC06F0A5
:1036F40000C04EF101C04FF102C050F103C051F1BE
:103704004EC100F04FC101F050C102F051C103F0AD
:10371400046A056A066A076A59EC08F0000ED8A420
:10372400010E006E0052D8B477D04EC100F04FC1E4
:1037340001F050C102F051C103F00BEC11F0000E86
:10374400046E031808E10450021805E1045001183E
:1037540002E10050000A60E1800E006E800E5319F1
:10376400005C02E15251010857E252C160F170EC71
:1037740008F000C004F001C005F002C006F003C068
:1037840007F04EC100F04FC101F050C102F051C129
:1037940003F090EC0CF05F0E046E700E056E090ED3
:1037A400066E810E076EFDEC0BF0010ED8B0000E14
:1037B400006E005206E0090E0101525F000E535BD9
:1037C40005D00101080E525F000E535B52C160F137
:1037D40070EC08F000C004F001C005F002C006F06F
:1037E40003C007F04EC100F04FC101F050C102F018
:1037F40051C103F090EC0CF00BEC11F000C054F14B
:1038040001C055F102C056F103C057F101014E6BDE
:103814004F6B506B516B38D04EC100F04FC101F06B
:1038240050C102F051C103F00BEC11F000C054F18F
:1038340001C055F102C056F103C057F154C100F064
:1038440055C101F056C102F057C103F0A7EC11F0C5
:1038540000C004F001C005F002C006F003C007F088
:103864004EC100F04FC101F050C102F051C103F04C
:10387400FBEC10F000C04EF101C04FF102C050F15A
:1038840003C051F1526B536B010E496F49510A0A3F
:1038940038E049C100F0000E016E026E036E00367E
:1038A40000900136023603360036009001360236A7
:1038B4000336F70E0024F66E550E0120F76E000E47
:1038C4000220F86E09006F00D4FF01F009006F00B8
:1038D400D4FF02F009006F00D4FF03F009006F0069
:1038E400D4FF04F00450575D08E10350565D05E130
:1038F4000250555D02E10150545D01E202D0492BB2
:10390400C5D749514725006E000E4821016E52511A
:1039140000265351012200504A5F01504B5B4DB7C2
:1039240004D04751481101E104D0010E4A5F000E52
:103934004B5B030E4C15006E4DC101F0000E0116D9
:103944000050011004E0010E4A5F000E4B5B4CA5D1
:1039540040D04CA315D04CA103D02D0E416F02D002
:103964002B0E416F6000E3F4E1FF6000E7F4E2FF37
:10397400600007F5E6FF384B392B584B592B0ED016
:103984004CA10CD06000E3F4E1FF6000E7F4E2FF37
:10399400200EE66E384B392B584B592B800E006E97
:1039A400800E4B19005C02E14A51000811E26000EC
:1039B400E3F4E1FF6000E7F4E2FF300EE66E384B1B
:1039C400392B584B592B010E4A5F000E4B5BE6D73F
:1039D40041D04CB71AD0800E006E800E4B19005C9B
:1039E40002E14A51000811E26000E3F4E1FF6000E3
:1039F400E7F4E2FF200EE66E384B392B584B592B77
:103A0400010E4A5F000E4B5BE6D74CA315D04CA1C8
:103A140003D02D0E426F02D02B0E426F6000E3F4F0
:103A2400E1FF6000E7F4E2FF60000BF5E6FF384BCE
:103A3400392B584B592B0ED04CA10CD06000E3F419
:103A4400E1FF6000E7F4E2FF200EE66E384B392B0D
:103A5400584B592B49C100F04907005253E049C162
:103A640000F0000E016E026E036E00360090013607
:103A74000236033600360090013602360336F70E5E
:103A84000024F66E550E0120F76E000E0220F86E2B
:103A940009006F00D4FF04F009006F00D4FF05F0A3
:103AA40009006F00D4FF06F009006F00D4FF07F08F
:103AB40054C100F055C101F056C102F057C103F0E2
:103AC40085EC0FF00A0E046E000E056E066E076E8E
:103AD40085EC0FF008C000F009C001F00AC002F044
:103AE4000BC003F0300E00266000E3F4E1FF600039
:103AF400E7F4E2FF600003F0E6FF384B392B584B44
:103B0400592BA8D7800E006E800E5319005C02E179
:103B14005251000811E26000E3F4E1FF6000E7F4B1
:103B2400E2FF300EE66E384B392B584B592B010E01
:103B3400525F000E535BE6D7800E000A006E800EC3
:103B44004819005C02E14751080803E2080E496F76
:103B540002D047C149F14951475F000E485B4953C0
:103B640003E14DB701D00CD06000E3F4E1FF600045
:103B7400E7F4E2FF2E0EE66E384B392B584B592BE7
:103B840049C160F170EC08F04EC104F04FC105F07A
:103B940050C106F051C107F0F5EC01F0E7EC0EF06E
:103BA40000C054F101C055F102C056F103C057F1F1
:103BB400495354E0490749C100F0000E016E026EFA
:103BC400036E00360090013602360336003600904C
:103BD400013602360336F70E0024F66E550E012028
:103BE400F76E000E0220F86E09006F00D4FF04F097
:103BF40009006F00D4FF05F009006F00D4FF06F040
:103C040009006F00D4FF07F054C100F055C101F062
:103C140056C102F057C103F085EC0FF00A0E046E92
:103C2400000E056E066E076E85EC0FF008C000F0FE
:103C340009C001F00AC002F00BC003F0300E0026E8
:103C44006000E3F4E1FF6000E7F4E2FF600003F0EA
:103C5400E6FF384B392B584B592BAAD747514811FB
:103C640011E06000E3F4E1FF6000E7F4E2FF300EEE
:103C7400E66E384B392B584B592B010E475F000E1B
:103C8400485BECD74CA71CD0800E006E800E4B19FD
:103C9400005C02E14A51000813E26000E3F4E1FF32
:103CA4006000E7F4E2FF200EE66E384B392B584BE8
:103CB400592B010E4A5F000E4B5B4A514B11EDE14B
:103CC400BFEF11F0C00E4C15016E4DC102F0000E95
:103CD4000216000E021802E1000E0118D8A49ED0AC
:103CE4004CA937D06000F7F4E9FF6000FBF4EAFF69
:103CF4006F00B8FF00F06F00B8FF01F0600003F040
:103D0400E9FF600007F0EAFF6F00B8FF54F16F00AD
:103D1400B8FF55F16F00B8FF56F16F00B8FF57F1C7
:103D24006000F7F4E9FF6000FBF4EAFF040EEE2400
:103D3400006E000EEE20016E6000F7F4E1FF6000FB
:103D4400FBF4E2FF600003F0E6FF600007F0E6FF2B
:103D54003DD06000F7F4E9FF6000FBF4EAFF6F0078
:103D6400B8FF00F06F00B8FF01F0600003F0E9FF56
:103D7400600007F0EAFF6F00B8FF00F06F00B8FFC3
:103D840001F0000E01BEFF0E026E036E00C054F17E
:103D940001C055F102C056F103C057F16000F7F4B9
:103DA400E9FF6000FBF4EAFF020EEE24006E000E51
:103DB400EE20016E6000F7F4E1FF6000FBF4E2FF27
:103DC400600003F0E6FF600007F0E6FF800E57197D
:103DD400006E800E005C08E1000E565D05E1000EE9
:103DE400555D02E1000E545D18E2030E4C13000E03
:103DF4004D13006A016A026A036A5451005E555108
:103E0400015A5651025A5751035A00C054F101C085
:103E140055F102C056F103C057F16CD04CA937D00C
:103E24006000F7F4E9FF6000FBF4EAFF6F00B8FFFD
:103E340000F06F00B8FF01F0600003F0E9FF6000DC
:103E440007F0EAFF6F00B8FF54F16F00B8FF55F1B7
:103E54006F00B8FF56F16F00B8FF57F16000F7F438
:103E6400E9FF6000FBF4EAFF040EEE24006E000E8E
:103E7400EE20016E6000F7F4E1FF6000FBF4E2FF66
:103E8400600003F0E6FF600007F0E6FF33D0600057
:103E9400F7F4E9FF6000FBF4EAFF6F00B8FF00F0FD
:103EA4006F00B8FF01F0600003F0E9FF600007F065
:103EB400EAFF6F00B8FF54F16F00B8FF55F1000E30
:103EC400566F576F6000F7F4E9FF6000FBF4EAFFF8
:103ED400020EEE24006E000EEE20016E6000F7F478
:103EE400E1FF6000FBF4E2FF600003F0E6FF600026
:103EF40007F0E6FF000E481902E1000E47190FE132
:103F0400000E006E571908E10050561905E10050E3
:103F1400551902E15451000A02E1474B482BC00EE7
:103F24004C15006E00C005F0BAD0010E496F49511E
:103F34000A0A38E049C100F0000E016E026E036EF9
:103F44000036009001360236033600360090013602
:103F540002360336F70E0024F66E550E0120F76E76
:103F6400000E0220F86E09006F00D4FF01F0090072
:103F74006F00D4FF02F009006F00D4FF03F00900C2
:103F84006F00D4FF04F00450575D08E10350565D00
:103F940005E10250555D02E10150545D01E202D099
:103FA400492BC5D78BD0010E496F4951080A38E017
:103FB40049C100F0000E016E026E036E00360090DF
:103FC40001360236033600360090013602360336D7
:103FD400890E0024F66E560E0120F76E000E0220A4
:103FE400F86E09006F00D4FF01F009006F00D4FFE0
:103FF40002F009006F00D4FF03F009006F00D4FF42
:1040040004F00450575D08E10350565D05E1025089
:10401400555D02E10150545D01E202D0492BC5D740
:104024004DD0010E496F49510C0A38E049C100F0E6
:10403400000E016E026E036E0036009001360236E9
:10404400033600360090013602360336160E00247D
:10405400F66E550E0120F76E000E0220F86E090070
:104064006F00D4FF01F009006F00D4FF02F00900D3
:104074006F00D4FF03F009006F00D4FF04F0045074
:10408400575D08E10350565D05E10250555D02E1BC
:104094000150545D01E202D0492BC5D70FD0055021
:1040A400000AD8B442D70550C00AD8B43ED7055048
:1040B400800AD8B478D70550400AB3E0800E006E69
:1040C400800E4819005C02E14751495D03E247C193
:1040D40049F10DD0800E4819006E800E005C02E19B
:1040E4004951475D04E249C147F1000E486F4A5106
:1040F4004B110EE0030E4C15006E4DC101F0000E85
:1041040001160050011004E0010E4A5F000E4B5BE3
:10411400800E4819006E800E4B19005C02E14A5172
:10412400475D05E247514A5F48514B5B02D04A6BF9
:104134004B6BC40E4C15016E4D51080B026E0250B0
:10414400080A02E1400E011808E14A514B1104E04B
:10415400010E4A5F000E4B5B1CD0C00E4C15016E65
:104164004D51080B026E0250080A02E1800E01183C
:1041740010E1800E006E800E4B19005C02E14A5182
:10418400020805E2020E4A5F000E4B5B02D04A6B46
:104194004B6B4CA569D04CA315D04CA103D02D0E6C
:1041A400436F02D02B0E436F6000E3F4E1FF600025
:1041B400E7F4E2FF60000FF5E6FF384B392B584B6C
:1041C400592B3BD04CA10DD06000E3F4E1FF60001B
:1041D400E7F4E2FF200EE66E384B392B584B592B8F
:1041E4002CD0C00E4C15016E4D51080B026E0250BE
:1041F400080A02E1800E011820E16000E3F4E1FF07
:104204006000E7F4E2FF300EE66E384B392B584B72
:10421400592B4CAB03D0580E446F02D0780E446F28
:104224006000E3F4E1FF6000E7F4E2FF600013F5EF
:10423400E6FF384B392B584B592B4A514B1113E09D
:104244006000E3F4E1FF6000E7F4E2FF300EE66EA5
:10425400384B392B584B592B010E4A5F000E4B5BE0
:104264004A514B11EDE182D04A514B1115E04CB744
:1042740013D06000E3F4E1FF6000E7F4E2FF200EF6
:10428400E66E384B392B584B592B010E4A5F000E02
:104294004B5B4A514B11EDE14CA315D04CA103D01B
:1042A4002D0E456F02D02B0E456F6000E3F4E1FF45
:1042B4006000E7F4E2FF600017F5E6FF384B392BA6
:1042C400584B592B0ED04CA10CD06000E3F4E1FF05
:1042D4006000E7F4E2FF200EE66E384B392B584BB2
:1042E400592BC00E4C15016E4D51080B026E025035
:1042F400080A02E1400E01180DE16000E3F4E1FF59
:104304006000E7F4E2FF300EE66E384B392B584B71
:10431400592B2CD0C00E4C15016E4D51080B026E5A
:104324000250080A02E1800E011820E16000E3F463
:10433400E1FF6000E7F4E2FF300EE66E384B392B04
:10434400584B592B4CAB03D0580E466F02D0780E05
:10435400466F6000E3F4E1FF6000E7F4E2FF600011
:104364001BF5E6FF384B392B584B592B800E006E4A
:10437400800E4819005C02E14751495D0DE260007E
:10438400E3F4E1FF6000E7F4E2FF300EE66E384B41
:10439400392B584B592BEAD747C100F048C101F0DB
:1043A400010E475F000E485B00500110D8B43FD1A6
:1043B400C00E4C15006E00C05AF11CD147C100F06C
:1043C40048C101F0000E48BFFF0E026E036E0036B6
:1043D400009001360236033600360090013602366C
:1043E4000336F70E0024F66E550E0120F76E000E0C
:1043F4000220F86E09006F00D4FF04F009006F007A
:10440400D4FF05F009006F00D4FF06F009006F0027
:10441400D4FF07F054C100F055C101F056C102F0B9
:1044240057C103F085EC0FF00A0E046E000E056E02
:10443400066E076E85EC0FF008C000F009C001F0AD
:104444000AC002F00BC003F0300E0024496FE1D023
:104454004CAB4AD047C100F048C101F0000E48BF40
:10446400FF0E026E036E00360090013602360336EC
:1044740000360090013602360336890E0024F66EAB
:10448400560E0120F76E000E0220F86E09006F0030
:10449400D4FF04F009006F00D4FF05F009006F0099
:1044A400D4FF06F009006F00D4FF07F054C100F0F8
:1044B40055C101F056C102F057C103F085EC0FF06D
:1044C4000F0E0016000E011602160316840E0024A9
:1044D400F66E570E0120F76E000E0220F86E0900EA
:1044E4006F00D4FF49F149D047C100F048C101F041
:1044F400000E48BFFF0E026E036E003600900136B8
:104504000236033600360090013602360336890E31
:104514000024F66E560E0120F76E000E0220F86E8F
:1045240009006F00D4FF04F009006F00D4FF05F008
:1045340009006F00D4FF06F009006F00D4FF07F0F4
:1045440054C100F055C101F056C102F057C103F047
:1045540085EC0FF00F0E0016000E0116021603165E
:10456400620E0024F66E570E0120F76E000E022034
:10457400F86E09006F00D4FF49F14BD047C100F039
:1045840048C101F0000E48BFFF0E026E036E0036F4
:1045940000900136023603360036009001360236AA
:1045A4000336160E0024F66E550E0120F76E000E2B
:1045B4000220F86E09006F00D4FF04F009006F00B8
:1045C400D4FF05F009006F00D4FF06F009006F0066
:1045D400D4FF07F054C100F055C101F056C102F0F8
:1045E40057C103F085EC0FF0070E0014496F300E2D
:1045F40049270FD05A51000AD8B4E0D65A51C00AFC
:10460400D8B4DCD65A51800AD8B422D75A51400AB9
:10461400B5E06000E3F4E1FF6000E7F4E2FF60006E
:1046240027F5E6FF384B392B584B592BB5D64CA7F9
:104634001CD0800E006E800E4B19005C02E14A51C2
:10464400000813E26000E3F4E1FF6000E7F4E2FF36
:10465400200EE66E384B392B584B592B010E4A5F0E
:10466400000E4B5B4A514B11EDE1BFEF11F058C105
:0846740000F059C101F0120031
:10467C00FC0E3F015E175E81010EAE6E7C6A7D6A98
:02468C0012001A
:10468E0038C113F139C114F13AC115F13BC116F11C
:10469E003CC117F13DC118F13EC119F13FC11AF1EC
:1046AE0040C121F141C122F142C123F143C124F1A4
:1046BE0044C11DF145C11EF146C11FF147C120F194
:0246CE001200D8
:0C46D0006F00A0F701F001C000F0120024
:1046DC000C6A0E6A0250D8A487EF23F001C002F0D6
:1046EC0000C001F0006A0E860250D8A487EF23F0B8
:1046FC0001C002F0016A0E960E880250D8B499EFF0
:10470C0023F00E50035ED8A4D8A09FEF23F0D890CE
:10471C0002BEA5EF23F0003601360236032E8EEFD3
:10472C0023F09FEF23F0010E0C6EC9EC00F0A9EF03
:10473C0023F0020E0C6ED9EC00F0A9EF23F0040E5E
:08474C000C6EBCEC00F0120041
:10475400A00E0101096F470E0A6F380E0B6F010E90
:104764000C6F3E01F86BF96BFA6BFB6BEC0EFD17EB
:08477400F889F885F88F1200A6
:10477C00160E0101606F616B130E626FFFEC10F08F
:10478C00170E0101606F010E616F250E626FFFEC59
:04479C0010F0120007
:1047A0003F0E010138153E01F16F80EC0FF0F881EA
:1047B0000000F8A101D0FDD76F00BCFB00F06F0036
:0647C000C0FB01F0120035
:1047C600010138510308D8A0386B39510308D8A025
:1047D600396BF00E3D01F217010138513D01F2131C
:1047E600300EF21339C100F000360090003600900A
:1047F60000360090003600900050F413F38F12003C
:1048060001013B6B6000E3F4E9FF6000E7F4EAFFB7
:104816006F00B8FF3AF13A51000A10E03AC160F170
:10482600EEEC0BF001013B2B3B513825E96E000EF7
:0E4836003921EA6E6F00B8FF3AF1EDD712009B
:104844002A0E0101366F010E376F25C138F126C1DA
:1048540039F127C13AF128C13BF129C13CF1360EA7
:104864003D6F010E3E6FBAEC11F000C034F101C08F
:1048740035F100502525E16E01502621E26EE66AED
:0A48840034C100F035C101F012004C
:10488E00600097F4E9FF60009BF4EAFF6F00B8FF49
:10489E0027F1000E0101286F000E286F000E281957
:1048AE0002E1200E271907E0000E281902E1090E79
:1048BE00271901E003D0254B262BE2D7296B2A6B53
:1048CE002B6B2C6B000E281902E12D0E271905E11A
:1048DE002B4B2C2B254B262B08D0000E281902E132
:1048EE002B0E271902E1254B262B600097F4E9FFCA
:1048FE0060009BF4EAFF6F00B8FF27F1000E286FEF
:10490E00000E286F27C160F1E2EC0BF0005219E0A7
:10491E0029C100F02AC101F00A0E046E000E056EC8
:10492E0064EC0CF0300E275D026E000E2859036EFB
:10493E0002500024296F035001202A6F254B262B8D
:10494E00D4D72B512C1108E029510008006E2AC132
:10495E0001F0000E015604D029C100F02AC101F069
:02496E00120035
:0C49700025C138F126C139F146DF1200E4
:10497C00600097F4E9FF60009BF4EAFFEE5215E04B
:10498C00600097F4E9FF60009BF4EAFF60009FF47D
:10499C00D9FF6000A3F4DAFFEE50DE1806E1010146
:1049AC00254B262B274B282BE3D7600097F4E9FFE8
:1049BC0060009BF4EAFF60009FF4D9FF6000A3F451
:1049CC00DAFFDE50EE5C006E016A000E015A120036
:1049DC00600097F4F6FF60009BF4F7FF60009FF413
:1049EC00F8FF09006F00D4FF00F0005216E06000E1
:1049FC0097F4F6FF60009BF4F7FF60009FF4F8FF5C
:104A0C0009006F00D4FF69F1EDEC00F0010E01011B
:0C4A1C002527000E26232723DBD71200DD
:044A280053DE120047
:0A4A2C00AC8E7E8E0C0E7E1212007E
:104A36000D0E0101696FEDEC00F00A0E0101696FC0
:064A4600EDEC00F012008F
:104A4C000050086E0150006E016A026A036A0B6A1C
:104A5C000C6A960E036E0A6A00C001F008C000F0E2
:084A6C00086A026A35DE12003F
:104A7400120E0101606F616B090E626FFFEC10F0A2
:044A8400FBDD120044
:104A8800AB50010F006E016A000E012225C104F02F
:104A980026C105F064EC0CF0060E046E00C002F0AE
:104AA80001C003F0045005E003320232039EFF0FF9
:104AB800FAD760000BF07CFF60000FF07DFF12005A
:104AC80009006F00D7FFE6FF0006FAE10106F8E1EA
:024AD8001200CA
:104ADA003901C06BC16BC26BCA6A3A01406B408331
:104AEA00830EC26E41934293C396C298C394BB8607
:104AFA00BA88BB84C296BA96506BCB6AFF0EC36E55
:104B0A00FF0E516F3E01BC6BB86BCC6A920EC46E3D
:104B1A003A01606B130E166F170EE56F3E01C16BFB
:084B2A00C19FC183C19112007B
:0C4B320010DE25C138F133DEF89F1200C0
:104B3E0025C102F026C103F002C000F003C001F04F
:104B4E00024A032A600003F0E9FF600007F0EAFF63
:104B5E00EE5201E0F1D701012551025C006E2651A3
:0E4B6E000358016E010E005E000E015A120087
:104B7C00FFDD280E0101386F4A0E396F000E3A6FB7
:104B8C00000E3B6FDA0E3C6F010E3D6F690E3E6FEF
:104B9C00010E3F6FFF0E406FFF0E416F000E426F14
:104BAC00000E436F5C0E446F010E456F000E466F96
:0E4BBC00000E476F66DD386B396BFFDD1200AF
:104BCA003C6A3D6A000E3D5C02E14F0E3C5C18E215
:104BDA00B20E3C24E16E000E3D20E26E6F0087FFAC
:104BEA00E1FF6F008BFFE2FFE66A010E3C24006ED4
:104BFA00000E3D20016E00C03CF001C03DF0E2D73E
:104C0A000001B26B3C6A3D6A3A6A3B6A346A356AA9
:104C1A000101116B126B046B3D01F289F96BFA6B9E
:084C2A003901A39793871200E2
:104C3200CBEC2BF051DF366A376A800E3718006EE4
:104C4200800E005C02E1200E365C10E28E0E3624ED
:104C5200E16E000E3720E26E6F0087FFE1FF6F000A
:104C62008BFFE2FFE66A364A372AE7D7366A376AA7
:104C7200800E3718006E800E005C02E1500E365C2A
:104C820010E23E0E3624E16E000E3720E26E6F0017
:104C920087FFE1FF6F008BFFE2FFE66A364A372AA1
:104CA200E7D73C6A3D6A346A356A3E0E2F6E000EC3
:104CB200306E080E3D01F56F020EF66FF28F5DDF6A
:104CC200280E0101386F4A0E396F000E3A6F000E3E
:104CD2003B6FDA0E3C6F010E3D6F690E3E6F010EA7
:104CE2003F6FFF0E406FFF0E416F000E426F000ECE
:104CF200436F5C0E446F010E456F000E466F000E4F
:104D0200476FC4DC0B0E0B6E260E0C6E5D0E0D6E25
:104D12000D2EFED70C2EFCD70B2EFAD7000000006A
:104D22000C0E696FEDEC00F085DE3E0E0101256F81
:104D3200570E266F000E276F50DE160E0101256FEB
:104D4200570E266F000E276F48DED30E0101256F26
:104D5200530E266F000E276F40DE540E0101256FA1
:104D6200530E266F000E276F38DE0E0E0101256FDF
:104D7200540E266F000E276F30DEE50E0101256FFF
:104D8200540E266F000E276F28DE2A0E0101256FB2
:104D9200570E266F000E276F20DE400E2D6E9C0EE2
:104DA2002E6E2FC025F130C026F1680E0101276F4B
:104DB200560E286F000E296F400E2A6F9C0E2B6F25
:104DC20040DD2FC025F130C026F1D1DD040E2B6E5F
:104DD200000E2C6E800E006E800E2C18005C02E11C
:104DE2002B50000823E2BC84060E0B6E130E0C6ED1
:104DF200AD0E0D6E0D2EFED70C2EFCD70B2EFAD754
:104E020000000000BC94060E0B6E130E0C6EAD0E6D
:104E12000D6E0D2EFED70C2EFCD70B2EFAD70000EE
:104E22000000010E2B5E000E2C5AD4D792DC010E2C
:104E32000101256F7DDE00C032F001C033F03194F4
:104E4200196A1A6AD28ED28C3901938F366A376AFE
:104E52000001AE6B460E0101256F550E266F000E46
:104E6200276FBBDDE40E0101256F560E266F000E83
:104E7200276FB3DD600EAC129C0EAB6EFADDA90E8D
:104E82000101256F560E266F000E276FA6DD330E29
:104E9200226E000E236EBA86330E0101256F000EBC
:104EA200266FF1DDC2DD060E0B6E130E0C6EAD0E1B
:104EB2000D6E0D2EFED70C2EFCD70B2EFAD700004E
:104EC2000000BA96470E0101256F540E266F000EA0
:104ED200276F83DDA10E0101256F550E266F000E8F
:104EE200276F7BDDCD0E0101256F550E266F000E5B
:104EF200276F73DD9FDD010E216E3C6A3D6A346AC5
:104F0200356A0101116B126B3901818B918BD28E43
:104F120001010F6B106B010E256F0ADE00C00DF14F
:104F220001C00EF12150010A1AE10DC100F00EC1BB
:104F320001F001320032019E01320032019E013243
:104F42000032019E01320032019E00C022F001C0F7
:104F520023F000C025F1000E0101266F94DD3E0E04
:104F62002F6E000E306E22C000F023C001F06DDD06
:104F7200390E046EB40E056E480E066E7D0E076E77
:104F8200F5EC01F000C005F101C006F102C007F125
:104F920003C008F12FC025F130C026F1940E0101A3
:104FA200276F530E286F000E296F36C02AF137C0C3
:104FB2002BF10DC12CF10EC12DF10DC12EF10EC13F
:104FC2002FF100C030F101C031F102C032F103C053
:104FD20033F137DC2FC025F130C026F1C8DC2ADDE1
:104FE200800E006E800E01011019005C02E10F516B
:104FF200000814E22FC025F130C026F1730E276F8E
:10500200570E286F000E296F0FC12AF110C12BF124
:1050120018DC2FC025F130C026F1A9DCD5DDBA8617
:10502200330E0B6EBB0E0C6EDF0E0D6E0D2EFED709
:105032000C2EFCD70B2EFAD700000000BA96000EF9
:105042000101121902E1010E1119D8A45BD13E0E21
:105052002F6E000E306E2FC025F130C026F1010EEA
:10506200276F570E286F000E296FB20E2A6F000E9F
:105072002B6F22EC24F02FC025F130C026F177DC13
:105082000001B251430AD8A4B4D0000E006E3550CC
:10509200005C02E134500108D8B0ABD0B30E01017C
:1050A200256F000E266F4ADD00C0B0F001C0B1F0DE
:1050B200010E366E000E376E800E3718006E800EAF
:1050C2000001B119005C02E1B051365C1CE2B20E83
:1050D2003624E96E000E3720EA6E6F00A7FFE9FF63
:1050E2006F00ABFFEAFF6F00B8FF00F000C0AFF047
:1050F200AFC060F1E2EC0BF00050000A01E103D016
:10510200364A372AD9D737500001B11902E1B051D6
:1051120036186FE1B30E0101256F000E266F47ECC2
:1051220024F000C0B0F001C0B1F0800E026E800E1B
:105132000118025C02E10050000819E2800E000131
:10514200B119006E800E010A005C02E1000EB05D32
:105152000EE2B0C022F0B1C023F0216A450E010177
:10516200256F560E266F000E276F37DC02D0226A9B
:10517200236ABA8622C025F1000E0101266F83DC64
:1051820022C000F023C001F060DC390E046EB40EC0
:10519200056E480E066E7D0E076EF5EC01F000C03E
:1051A20005F101C006F102C007F103C008F1250EA6
:1051B2000101046F2FC025F130C026F1750E276F53
:1051C200550E286F000E296F22C02AF123C02BF141
:1051D20000C02CF101C02DF102C02EF103C02FF14D
:1051E20022EC24F02FC025F130C026F1B8EC24F0D7
:1051F200BA960001B251410A13E1000E006E355019
:10520200005C02E1345000080BE2010E216E1F0E19
:105212000101256F560E266F000E276FEEEC24F06B
:105222000001AF6BB20E0101256F000E266F1B0E3F
:10523200276F000E286FBEEC24F000C002F101C0FF
:1052420003F1000E011802E1000E001858E10001FE
:10525200B06BB16B800EB119006E800E005C02E182
:10526200FE0EB05D1BE2B0C038F0B1C039F0B0C084
:1052720025F1B1C026F107DC020E0B6E450E0C6E55
:10528200A90E0D6E0D2EFED70C2EFCD70B2EFAD7C3
:10529200000000000001B04BB12BDCD7FF0EB06F55
:1052A200000EB16F800E006E800EB119005C02E13B
:1052B200B05101081EE2B0C038F0B1C039F0B0C040
:1052C20025F1B1C026F144EC25F0020E0B6E450E1D
:1052D2000C6EA90E0D6E0D2EFED70C2EFCD70B2ECA
:1052E200FAD700000000010E0001B05F000EB15BB2
:1052F200D9D722C025F123C026F144EC25F00101C3
:10530200116B126B000E121902E1020E11191CE14F
:105312003E0E2F6E000E306E2FC025F130C026F1EA
:10532200C70E276F560E286F000E296F34C02AF160
:1053320035C02BF122EC24F02FC025F130C026F12C
:10534200B8EC24F0116B126B364A372ABA78E3D5DF
:02535200FFD783
:1057960010EE19F0120E006E010E016E500EF66E2E
:0E57A600570EF76E000EF86E64EC25F0120040
:105354002050726F6A6574203A2031384632374BD8
:1053640034325F426173655F55415254315F525824
:105374005F49545F414443305F50574D5F38626921
:1053840074735F323032312E6D637070690D0A00B0
:10539400204D65737572652023253564203D3E20BC
:1053A40041444320524131203D20202520356420B2
:1053B40020736F6974202530345820204475747923
:0F53C400204379636C653D25332E316625250026
:1053D300204469726563746F7279203A20433A5CA2
:1053E3005F4D696B726F435C5F4D657350726F6A9B
:1053F3006574735F4D696B726F435C5F313846321E
:0B540300374B34325F50574D0D0A004C
:10540E0020536F75726365203A205F31384632370C
:10541E004B34325F33324D687A5F55617274315F4F
:10542E004144435F50574D5F38625F323032312D09
:09543E00303931322E630D0A00F1
:1054470020636465204120706F75722044757479FC
:10545700206379636C65207265676CE920706172FF
:1054670020706F7461722028414E414C4F4749515B
:065477005545290D0A0055
:10547D000000007FCDCC4C7B0AD723786F120375CB
:10548D0017B75171ACC5276EBD37066B95BF566703
:10549D0077CC2B645F700961FFE65B5D08E53C3CF2
:0454AD006042221B1C
:1054B1000000007F000020820000488500007A88FB
:1054C10000401C8C0050438F0024749280961896E3
:1054D10020BC3E99286B6E9CF90215A0EC782DC179
:0454E100CAF249E2E0
:1054E50020434F4E464947203A20503138463237FF
:1054F5004B34325F464F53435F5131304D487A78D4
:10550500345F34304D487A2E6366677363680D0ADD
:015515000095
:10551600010000000800000040000000000200003A
:1055260000100000008000000000040000002000C1
:10553600000000010000000800000040000000001C
:1055460020536F727469652050574D31204166664D
:10555600656374E9652070617220646566617574BF
:0F556600207375722050494E205243320D0A00B7
:10557500204E65772049526174696F202838206272
:1055850069747329203D202535642020736F697463
:0C5595002025332E31662025250D0A004C
:1055A1002049526174696F2061646A757374E920DE
:1055B10076696120506F742E416E616C6F67207047
:0C55C10061722064E9666175740D0A00D7
:1055CD002063646520437878782020706F75722091
:1055DD0044757479206379636C6520766961204B1D
:0A55ED004559424F4152440D0A0097
:1055F700010000000A00000064000000E80300004A
:1056070010270000A086010040420F0080969800F6
:0856170000E1F50500CA9A3B11
:10561F000D0A2049726174696F2061646A75737431
:10562F0020627920416E616C6F67206D6F64652019
:06563F006E6F770D0A00FA
:105645000D0A2049726174696F2061646A7573740B
:10565500206279204B6579626F617264206E6F7785
:035665000D0A002B
:1056680020436C6F636B20696E697469616C652097
:10567800696E204B687A203D2025303575200D0A4B
:015688000021
:1056890001000000100000000001000000100000EF
:1056990000000100000010000000000100000010DF
:1056A90020496E69742049526174696F20E0203283
:0E56B900302520736F6974203531200D0A00F2
:1056C70042756666657231205541525431204675E0
:0D56D7006C6C203D2025303564200D0A004C
:1056E40020496E69742050574D31203862697473B3
:0D56F4002061742031303030487A0D0A00FA
:10570100205265636570742055415254313D202506
:0557110073200D0A00E9
:1057160020506F77657220737570706C793A2035FA
:04572600560D0A0012
:10572A0020464F534320203A205131304D487A7851
:04573A00340D0A0020
:10573E00204D4355203A2031384632374B34320D06
:02574E000A004F
:02575000000057
:0657520052414D504500DC
:015758000050
:0257590000004E
:07575B00286E756C6C29003B
:1057620030313233343536373839616263646566D5
:015772000036
:105773002020657272657572203D202535640D0AFF
:015783000025
:105784003031323334353637383941424344454673
:015794000014
:020000040030CA
:0A000000220925A70B3F9F0F010006
:00000001FF
